:020000001129C4
:100008000408A2008316071383120930A300031003
:100018001420A20CA30B0C280314142003140C297D
:1000280003181928000007135528071755282C0806
:10003800A0002D08A100A201A3018316871783122F
:10004800252826286400871F4228FF30A207031CA2
:10005800A307031CA007031CA107031C0C29220FDC
:100068002428230F2528FA30A2000030A3002628D0
:100078008316871783126400871B3F280030A1006E
:100088001930DC200830A30055200310871B031407
:10009800A20C00004F28A30B48285520031422085F
:1000A80008000030A1006630DC28A401A501B512C3
:1000B8000721031C0800D33E0319B5162D3EC63E82
:1000C80003186A280A3E031C5C287128F33E0318AB
:1000D8005C28063E031C5C280A3EA2000430A300EC
:1000E8000310A40DA50DA30B74282208A404A903CA
:1000F800031990280721031C0800C63E0318882806
:100108000A3E031C90287128F33E03189028063EE7
:10011800031C90280A3E7128B51E9728A409A50932
:10012800A40A0319A50A240803140C29B5132908DD
:100138000319B5170430A800250EA7202508A72005
:10014800240EA72024080F39F63E0318073E0A3E5E
:10015800CA28B51329080319B5170530A800273090
:10016800A3001030C3200330A300E830C320A3014C
:100178006430C320A3010A30C3202408CA28A2007F
:100188002508A1002408A000EB202008A000A8034F
:100198000319B51329080319D428280203180800DD
:1001A8002008031DB513B51B0800303E0729A1011F
:1001B800FC3EA000A109031CE728FF300000A007AF
:1001C8000318E228A0076400A10FE1280800A50190
:1001D800A4011030A600210DA40DA50D2208A4022B
:1001E8002308031C230FA502031801292208A407CA
:1001F80023080318230FA5070310A00DA10DA60BB4
:10020800EF2820080C29840031088A003008820071
:10021800831303138312640008000D308A0105203C
:100228000A308A01052053308A01052074308A017A
:10023800052061308A01052072308A01052074305A
:100248008A01052069308A0105206E308A0105205F
:1002580067308A0105202E308A0105202E308A0158
:1002680005200D308A0105200A308A0105208A11EF
:100278000A1289293C084007C4003D080318013EBA
:100288004107C50003184614031C46103A083E07E8
:10029800B2003B080318013E3F07B30003014618AC
:1002A80001303207C20033080318013EC3000800BA
:1002B80040083C02C4004108031C013E3D02C50041
:1002C80003184614031C461064008A110A12461CBF
:1002D80078293E083A02C2003F08031C013E3B024F
:1002E800C3008A110A1288293E083A02B2003F0860
:1002F800031C013E3B02B30001303202C200003051
:10030800031C013E3302C30008000A308A0105209D
:100318000D308A01052044308A01052045308A01C4
:1003280005204D308A0105204F308A0105202030F4
:100338008A0105206F308A01052066308A01052070
:1003480020308A01052033308A01052032308A01A5
:10035800052020308A01052062308A010520693095
:100368008A01052074308A01052020308A01052081
:1003780069308A0105206E308A01052073308A01B0
:10038800052069308A01052067308A0105206E3012
:100398008A01052065308A01052064308A0105201C
:1003A80020308A01052041308A01052064308A0105
:1003B800052064308A01052069308A0105207430DF
:1003C8008A01052069308A0105206F308A010520DD
:1003D8006E308A01052020308A01052026308A01E6
:1003E800052020308A01052053308A010520753008
:1003F8008A01052062308A01052074308A010520AF
:1004080072308A01052061308A01052063308A0133
:10041800052074308A01052069308A0105206F3073
:100428008A0105206E308A0105200D308A010520D9
:100438000A308A01052033308A01052032308A01CA
:10044800052062308A01052069308A010520743050
:100458008A01052020308A01052076308A0105208E
:1004680061308A0105206C308A01052075308A01C7
:10047800052065308A01052073308A0105203A304D
:100488008A01052020308A0105204E308A01052086
:1004980075308A0105206D308A01052031308A01C6
:1004A800052020308A0105203D308A0105202030B2
:1004B8008A01052032308A01052032308A01052060
:1004C80033308A01052034308A01052035308A010D
:1004D800052036308A01052037308A01052038305A
:1004E8008A01052039308A01052030308A0105202B
:1004F80020308A01052028308A01052064308A01CD
:10050800052065308A01052063308A0105202930DD
:100518008A01052020308A0105203D308A01052006
:1005280020308A01052038308A01052035308A01BB
:10053800052033308A01052030308A0105204330F8
:100548008A01052043308A01052044308A010520AC
:1005580032308A01052020308A01052028308A019E
:10056800052068308A01052065308A010520783029
:100578008A01052029308A0105200D308A010520CD
:100588000A308A01052020308A01052020308A019E
:10059800052020308A01052020308A0105202030DE
:1005A8008A01052020308A01052020308A01052093
:1005B80020308A01052020308A01052020308A0158
:1005C800052020308A01052020308A0105202030AE
:1005D8008A01052020308A0105204E308A01052035
:1005E80075308A0105206D308A01052032308A0174
:1005F800052020308A0105203D308A010520203061
:100608008A01052031308A01052030308A01052011
:1006180039308A01052038308A01052037308A01AF
:10062800052036308A01052035308A01052034300E
:100638008A01052033308A01052032308A010520DD
:1006480020308A01052028308A01052064308A017B
:10065800052065308A01052063308A01052029308C
:100668008A01052020308A0105203D308A010520B5
:1006780020308A01052034308A01052031308A0172
:10068800052037308A01052044308A01052044308E
:100698008A01052034308A01052037308A01052077
:1006A80038308A01052020308A01052028308A0147
:1006B800052068308A01052065308A0105207830D8
:1006C8008A01052029308A0105200D308A0105207C
:1006D8000A308A0105203030BA008530BB00D2309C
:1006E800BC00CC30BD007D30BE004130BF0078304A
:1006F800C000D430C1000D308A0105200A308A01BB
:10070800052043308A01052061308A0105206C30BC
:100718008A01052063308A01052075308A01052089
:100728006C308A01052061308A01052074308A0105
:10073800052065308A01052064308A0105202030B3
:100748008A01052072308A01052065308A0105205A
:1007580073308A01052075308A0105206C308A01C2
:10076800052074308A01052073308A0105203A304B
:100778008A0105200D308A0105200A308A010520EA
:100788008A110A12FF2E0A308A0105200D308A01CB
:10079800052059308A0105206F308A0105207530FF
:1007A8008A01052020308A01052063308A0105204E
:1007B80061308A0105206E308A01052020308A01C7
:1007C800052074308A01052072308A0105207930AD
:1007D8008A01052020308A01052069308A01052018
:1007E80074308A01052020308A01052062308A0190
:1007F800052079308A01052020308A0105206530DE
:100808008A0105206E308A01052074308A0105208E
:1008180065308A01052072308A01052069308A0115
:1008280005206E308A01052067308A0105202030B6
:100838008A01052074308A01052077308A01052055
:100848006F308A01052020308A01052033308A0163
:10085800052032308A01052062308A01052069307E
:100868008A01052074308A01052020308A0105207C
:100878006E308A01052075308A0105206D308A01A5
:10088800052062308A01052065308A010520723012
:100898008A01052073308A01052020308A0105204D
:1008A80061308A01052073308A01052020308A01D1
:1008B800052068308A01052065308A0105207830D6
:1008C8008A01052020308A01052076308A0105201A
:1008D80061308A0105206C308A01052075308A0153
:1008E800052065308A01052073308A0105200D3006
:1008F8008A0105200A308A01052054308A01052022
:1009080068308A01052065308A01052020308A0177
:10091800052066308A01052069308A010520723079
:100928008A01052073308A01052074308A01052068
:1009380020308A0105206E308A01052075308A0131
:1009480005206D308A01052062308A010520653056
:100958008A01052072308A01052020308A0105208D
:1009680073308A01052068308A0105206F308A01BA
:10097800052075308A0105206C308A010520643015
:100988008A01052020308A01052062308A0105206D
:1009980065308A01052020308A01052074308A01DB
:1009A800052068308A01052065308A01052020303D
:1009B8008A0105206F308A0105206E308A010520E2
:1009C80065308A01052020308A01052077308A01A8
:1009D800052069308A01052074308A0105206830B5
:1009E8008A01052020308A01052074308A010520FB
:1009F80068308A01052065308A01052020308A0187
:100A0800052068308A01052069308A010520673091
:100A18008A01052068308A01052065308A01052091
:100A280072308A01052020308A01052076308A013B
:100A3800052061308A0105206C308A010520753057
:100A48008A01052065308A0105200D308A010520BC
:100A58000A308A01052045308A0105206E308A0156
:100A6800052074308A01052065308A01052072301E
:100A78008A01052020308A01052061308A0105207D
:100A880020308A0105207E308A01052020308A0125
:100A9800052028308A01052074308A010520693034
:100AA8008A0105206C308A01052064308A010520FE
:100AB80065308A01052029308A01052020308A0105
:100AC800052074308A0105206F308A010520203006
:100AD8008A01052062308A01052065308A010520D7
:100AE80067308A01052069308A0105206E308A0145
:100AF80005202E308A0105202E308A0105202E304F
:100B08008A0105202E308A0105202E308A01052011
:100B18000D308A0105200A308A0105208A013C200F
:100B28007E3C8A110A12031D922D0D308A01052080
:100B38000A308A01052045308A0105206E308A0175
:100B4800052074308A01052065308A01052072303D
:100B58008A01052020308A0105204E308A010520AF
:100B680075308A0105206D308A01052031308A01EF
:100B7800052020308A01052061308A010520733064
:100B88008A01052020308A01052061308A0105206C
:100B980020308A01052068308A01052069308A01E1
:100BA800052067308A01052068308A010520203039
:100BB8008A01052077308A0105206F308A010520D7
:100BC80072308A01052064308A01052020308A01AC
:100BD800052061308A0105206E308A0105206430C5
:100BE8008A01052020308A0105206C308A01052001
:100BF8006F308A01052077308A01052020308A016C
:100C0800052077308A0105206F308A01052072306F
:100C18008A01052064308A01052020308A010520D8
:100C280069308A0105206E308A01052020308A014A
:100C3800052068308A01052065308A010520783052
:100C48008A0105200D308A0105200A308A01052015
:100C58002030AC004E30AD000430A9001B30B0008D
:100C6800B1018A0159208A110A12031CC72BBA0044
:100C78002508BB000430A9001B30B000B1018A016F
:100C880059208A110A12031CC72BBC002508BD0075
:100C98000D308A0105200A308A01052045308A0175
:100CA80005206E308A01052074308A0105206530E0
:100CB8008A01052072308A01052020308A0105202A
:100CC8004E308A01052075308A0105206D308A0171
:100CD800052032308A01052020308A010520613044
:100CE8008A01052073308A01052020308A010520F9
:100CF80061308A01052020308A01052068308A0188
:100D0800052069308A01052067308A01052068308E
:100D18008A01052020308A01052077308A010520C4
:100D28006F308A01052072308A01052064308A01FB
:100D3800052020308A01052061308A0105206E30A7
:100D48008A01052064308A01052020308A010520A7
:100D58006C308A0105206F308A01052077308A01BE
:100D6800052020308A01052077308A0105206F3060
:100D78008A01052072308A01052064308A01052025
:100D880020308A01052069308A0105206E308A01E9
:100D9800052020308A01052068308A010520653049
:100DA8008A01052078308A0105200D308A01052046
:100DB8000A308A0105202030AC004E30AD000430E6
:100DC800A9001B30B000B1018A0159208A110A120A
:100DD800031CC72BBE002508BF000430A9001B3028
:100DE800B000B1018A0159208A110A12031CC72BCD
:100DF800C0002508C1008A013E210D308A01052066
:100E08000A308A01052041308A01052044308A01D0
:100E1800052044308A01052049308A0105205430D4
:100E28008A01052049308A0105204F308A010520B2
:100E38004E308A01052020308A01052052308A016F
:100E4800052065308A01052073308A010520753038
:100E58008A0105206C308A01052074308A0105203A
:100E680020308A01052069308A0105206E308A0108
:100E7800052020308A01052068308A010520653068
:100E88008A01052078308A0105203A308A01052038
:100E980020308A0105200430A9004208A400430834
:100EA800A5000430B000B1018A019A200430A900DD
:100EB8004408A4004508A5000430B000B1018A0127
:100EC8009A2020308A01052028308A0105204330E5
:100ED8008A01052061308A01052072308A010520C7
:100EE80072308A01052079308A01052020308A0174
:100EF800052062308A01052069308A010520743096
:100F08008A0105203D308A010520A90100304618D4
:100F18000130A400A5010430B000B1018A01AD2060
:100F280029308A0105200A308A0105200D308A01FE
:100F380005208A015C210D308A0105200A308A01CA
:100F4800052053308A01052055308A01052042309A
:100F58008A01052054308A01052052308A01052073
:100F680041308A01052043308A01052054308A0126
:100F7800052049308A0105204F308A0105204E306E
:100F88008A01052020308A01052052308A01052077
:100F980065308A01052073308A01052075308A0181
:100FA80005206C308A01052074308A010520203024
:100FB8008A01052069308A0105206E308A010520E2
:100FC80020308A01052068308A01052065308A01B1
:100FD800052078308A0105203A308A010520203022
:100FE8008A0105200430A9004208A4004308A5008E
:100FF8000430B000B1018A019A200430A9004408E5
:10100800A4004508A5000430B000B1018A019A2067
:1010180020308A01052028308A01052043308A01C2
:10102800052061308A01052072308A01052072305E
:101038008A01052079308A01052020308A0105209F
:1010480062308A01052069308A01052074308A01DE
:1010580005203D308A010520A901003046180130DD
:10106800A400A5010430B000B1018A01AD202930E7
:101078008A0105200A308A0105200D308A010520E1
:0C1088008A01C72B63008A150A12462853
:02400E00753FFC
:00000001FF
